:02000000162FB9
:08000800FF00030E8312031335
:10001000C8000A0EC900040ECA008A110A123E2F37
:10002000E208031D14280800F930FF3E031D1528BF
:100030000000E20B1428080000000000000000008F
:10004000000000000000EE0B1C2808000330DE0753
:10005000DE0CDE0C7F30DE050000DE0B2C280800F5
:10006000F301F401F501F601F801F901FA01FB01D0
:10007000F701F71A08000310F80DF90DFA0DFB0D42
:1000800083120313EB0DEC0DED0DEE0DF30DF40DDE
:10009000F50DF60D72087602031D582871087502D9
:1000A000031D582870087402031D58286F08730236
:1000B000031C69286F08F3027008031C700FF40218
:1000C0007108031C710FF5027208031C720FF6020F
:1000D0007814F70A3928EB01EC01EE01EF01ED018C
:1000E0006D1A08000310EE0DEF0DE50DE60DEB0D9A
:1000F000EC0D68086C02031D7F2867086B02031C67
:1001000088286708EB026808031CEC03EC026E14F5
:10011000ED0A7028E101600861020318080064001C
:100120000130E2001020E10A8B28861006118611AA
:100130008613861206126B0E0F39ED000F30ED0597
:100140006D188614ED1806156D198615ED198617AC
:10015000EC08031D86160A30EE001C2006160A3035
:10016000EE001C2006120F306B05ED000A30EE0089
:100170001C208610061186118613861206126D1831
:100180008614ED1806156D198615ED198617EC08FD
:10019000031D86160A30EE001C2006160A30EE00FB
:1001A0001C2006120A30EE001C200800EC01ED01B4
:1001B000EE01EF01F001EC1A0800641CED28600864
:1001C000ED0761080318610FEE0762080318620F5C
:1001D000EF0763080318630FF0070310E70CE60C42
:1001E000E50CE40C0310E00DE10DE20DE30DEC0A6B
:1001F000DB28EB01EC015E08E9005F08EA00E7019B
:100200006008E8006108E7046B08E7046C08E8048C
:100210006708E2006808E3006908E4006A08E5008E
:1002200000306A02031D1E2998306902031D1E2931
:1002300096306802031D1E2980306702031C552971
:100240006208EB006308EC006408ED006508EE004E
:100250008030EF009630F0009830F1000030F2006E
:100260003020780883120313E6006608303EEB0066
:100270001030EC0095206608003C031855298030AA
:10028000E202E308E408E5089630EB00031C6B0F7C
:10029000E3029830EB00031C6B0FE4020030EB002C
:1002A000031C6B0FE502E6033B2900306A02031DC5
:1002B00063290F306902031D632942306802031D60
:1002C000632940306702031C9F296208EB00630822
:1002D000EC006408ED006508EE004030EF004230AD
:1002E000F0000F30F1000030F20030207808831267
:1002F0000313E6006608303EEB001030EC0095205A
:100300002E30EB001030EC0095206608003C0318FE
:100310009F294030E202E308E408E5084230EB00A0
:10032000031C6B0FE3020F30EB00031C6B0FE402A6
:100330000030EB00031C6B0FE502E603852900305B
:100340006A02031DAD2901306902031DAD29863003
:100350006802031DAD29A0306702031CE42962086E
:10036000EB006308EC006408ED006508EE00A030C7
:10037000EF008630F0000130F1000030F200302054
:10038000780883120313E6006608303EEB00103055
:10039000EC0095206608003C0318E429A030E20236
:1003A000E308E408E5088630EB00031C6B0FE3026A
:1003B0000130EB00031C6B0FE4020030EB00031C68
:1003C0006B0FE502E603CA2900306A02031DF22919
:1003D00000306902031DF22927306802031DF2294B
:1003E00010306702031C272A6208EB006308EC0048
:1003F0006408ED006508EE001030EF002730F000D3
:10040000F101F2013020780883120313E600660838
:10041000303EEB001030EC0095206608003C0318DD
:10042000272A1030E202E308E408E5082730EB0051
:10043000031C6B0FE3020030EB00031C6B0FE402A4
:100440000030EB00031C6B0FE502E6030D2A0030C1
:100450006A02031D352A00306902031D352A033064
:100460006802031D352AE8306702031C6F2A620800
:10047000EB006308EC006408ED006508EE00E8306E
:10048000EF000330F000F101F20130207808831210
:100490000313E6006608303EEB001030EC009520B8
:1004A0002E30EB001030EC0095206608003C03185D
:1004B0006F2AE830E202E308E408E5080330EB00C5
:1004C000031C6B0FE3020030EB00031C6B0FE40214
:1004D0000030EB00031C6B0FE502E603552A0030E9
:1004E0006A02031D7D2A00306902031D7D2A003047
:1004F0006802031D7D2A64306702031CB12A62086A
:10050000EB006308EC006408ED006508EE00643061
:10051000EF00F001F101F20130207808831203139B
:10052000E6006608303EEB001030EC0095206608CF
:10053000003C0318B12A6430E202E308E408E5084D
:100540000030EB00031C6B0FE3020030EB00031CD8
:100550006B0FE4020030EB00031C6B0FE502E603B7
:10056000972A00306A02031DBF2A00306902031D6A
:10057000BF2A00306802031DBF2A0A306702031C2D
:10058000F32A6208EB006308EC006408ED006508DC
:10059000EE000A30EF00F001F101F201302078089E
:1005A00083120313E6006608303EEB001030EC00C7
:1005B00095206608003C0318F32A0A30E202E3089B
:1005C000E408E5080030EB00031C6B0FE302003089
:1005D000EB00031C6B0FE4020030EB00031C6B0FFD
:1005E000E502E603D92A3030EB006208EB07103051
:1005F000EC0095200800E501E50164086502031898
:10060000080083135F1883175E086507840080085D
:100610000319080083135F1883175E0865078400B9
:100620000008EB001030EC009520E50AFD2AE11FE0
:10063000262B2D30EB001030EC0095206008003C9C
:10064000E500E1090318E10A6508E0006008E2003E
:100650006108E30027306102031D302B1030600277
:10066000031C5E2BE11B5E2BE9016208E5006308B9
:10067000E600E31F412BE509E609E50A0319E60A4E
:10068000E90A1030E7002730E8006B206E08E4002C
:10069000691C4C2BE409E40A6408303EEB0010307E
:1006A000EC0095206408003C03185E2B1030E20239
:1006B0002730031C2830E302E403522B033061028D
:1006C000031D642BE8306002031C942BE11B942B68
:1006D000EA016208E5006308E600E31F752BE509FF
:1006E000E609E50A0319E60AEA0AE830E7000330FA
:1006F000E8006B206E08E9006A1C802BE909E90A12
:100700006908E4006408303EEB001030EC009520EE
:100710006408003C0318942BE830E2020330031C09
:100720000430E302E403882B6108803AE50080305E
:100730006502031D9D2B64306002031CC92BEA0176
:100740006208E5006308E600E31FAC2BE509E60953
:10075000E50A0319E60AEA0A6430E700E8016B20BB
:100760006E08E9006A1CB62BE909E90A6908E40089
:100770006408303EEB001030EC0095206408003C2B
:100780000318C92B6430E202E308031CE303E4030B
:10079000BE2B6108803AE50080306502031DD22B34
:1007A0000A306002031CFE2BEA016208E5006308C0
:1007B000E600E31FE12BE509E609E50A0319E60A6D
:1007C000EA0A0A30E700E8016B206E08E9006A1CBB
:1007D000EB2BE909E90A6908E4006408303EEB0004
:1007E0001030EC0095206408003C0318FE2B0A3002
:1007F000E202E308031CE303E403F32B6208303E48
:10080000EB001030EC0095200800DF08031D0B2CD6
:100810008030DF000D2CC030DF005E085F07EB008A
:10082000EC0195200230E0008A2008006008EB000F
:100830001030EC0095200800013083120313EB0008
:10084000EC0195200230E0008A200230EB00EC0140
:1008500095200230E0008A200800831603138610DA
:1008600083128610831606118312061183168611D1
:1008700083128611831686138312861383168612BB
:100880008312861283160612831206120C30E000C1
:100890008A203330EB00EC0195200230E0008A2002
:1008A0003330EB00EC0195200230E0008A2032303A
:1008B000EB00EC0195200230E0008A202C30EB00A8
:1008C000EC0195200230E0008A200630EB00EC01BC
:1008D00095200230E0008A200C30EB00EC019520DE
:1008E0000230E0008A200130EB00EC01952002305C
:1008F000E0008A200230EB00EC0195200230E0009D
:100900008A2008000730831203139F00C03083162B
:1009100081002D2483160610A73081008312CD019B
:10092000CE01D90181010B11831606148312DB015C
:1009300012305B020318BB2CDC01F2305C0203189E
:10094000B62C4630DD00DD0BA32C000000000000BB
:100950000B1DAF2C0B11CD0A0319CE0AB42C0000CD
:100960000000000000000000DC0A9D2C7030DE005A
:100970002620DB0A982C0000000000000000000088
:100980000000000000000000000000000B1DCD2C46
:100990000B11CD0A0319CE0AD22C00000000000072
:1009A000000000008316061083120108DA00FE30F2
:1009B000831606058600FE3083120605DF0001302F
:1009C0005F048600FE30831606058600FE30831223
:1009D000060586005903D9000108D800DE015A082F
:1009E0005802031DDE0ADE080319D72C0B11013053
:1009F000DE00DF0105241C2459030319D901463008
:100A0000E00016242030E00016243D30E0001624DB
:100A10002030E00016244D08DE004E08DF005A08A2
:100A2000E0005908E100F9202030E0004830E10002
:100A30007A30E200E3010030DF006030DE00033096
:100A4000E400FB224D08C4004E08C500C601C701E2
:100A5000CE1F2C2DC603C703DE015A08E9005E082D
:100A60005907E8000318E90AEA01EB014408E0002D
:100A70004508E1004608E2004708E300FF30E400D3
:100A8000E500E601E701D6206D08B4006E08B50068
:100A90006F08B6007008B7006808B4076908031843
:100AA000690FB5076A0803186A0FB6076B080318C1
:100AB0006B0FB707DE010130DF0005243708003C6B
:100AC000031D6C2D3608003C031D6C2D3508003CC1
:100AD000031D6C2D3408013C031C8A2D6E30E00090
:100AE00016246F30E00016242030E0001624733006
:100AF000E00016246930E00016246730E000162478
:100B00006E30E00016246130E00016246C30E00006
:100B100016248E2C5430E00016242030E0001624D9
:100B20003D30E00016242030E00016240030EB00B9
:100B3000CA30EC009A30ED003B30EE003408EF0094
:100B40003508F0003608F1003708F2003020780848
:100B500083120313B8007908B9007A08BA007B0839
:100B6000BB003B08003C031DBF2D3A080F3C031D92
:100B7000BF2D3908423C031DBF2D3808403C0318E7
:100B80004B2E3808EB003908EC003A08ED003B0822
:100B9000EE00E830EF000330F000F101F201302008
:100BA000780883120313B8007908B9007A08BA00EC
:100BB0007B08BB003808EB003908EC003A08ED0070
:100BC0003B08EE00E830EF000330F000F101F201E5
:100BD0003020780883120313BC007908BD007A081E
:100BE000BE007B08BF003C08E0003D08E1003E0875
:100BF000E2003F08E300E830E4000330E500E601EE
:100C0000E701D6206D08DE006E08E8006F08E900F5
:100C10007008EA005E083802C0003908C1003A08CE
:100C2000C2003B08C3006808031C680FC1026908C2
:100C3000031C690FC2026A08031C6A0FC3023C0846
:100C4000E0003D08E10017232C30E00016244008A6
:100C5000E0004108E10017232030E00016246D3049
:100C6000E00016247330E00016242030E000162443
:100C70002030E00016242030E00016242030E00070
:100C800016242030E00016242030E0001624203006
:100C9000E00016248E2CDF0100303B02031D5A2E8B
:100CA00000303A02031D5A2E03303902031D5A2E1A
:100CB000E93038020318DF0ADE0100303B02031D71
:100CC0006B2E0F303A02031D6B2E42303902031D8A
:100CD0006B2E40303802031CDE0A5E085F050319E4
:100CE000E22E3808EB003908EC003A08ED003B082A
:100CF000EE00E830EF000330F000F101F2013020A7
:100D0000780883120313BC007908BD007A08BE007E
:100D10007B08BF003C08E0003D08E1003E08E2001F
:100D20003F08E300E830E4000330E500E601E701B6
:100D3000D6206D08E8006E08E9006F08EA00700828
:100D4000EB0068083802C0003908C1003A08C20048
:100D50003B08C3006908031C690FC1026A08031C31
:100D60006A0FC2026B08031C6B0FC3023C08E00051
:100D70003D08E10017232C30E00016244008E00075
:100D80004108E10017232030E00016246D30E00018
:100D900016246B30E00016247330E0001624203057
:100DA000E00016242030E00016242030E000162455
:100DB0002030E00016242030E00016242030E0002F
:100DC00016248E2C3B08003C031DF02E3A08003CF4
:100DD000031DF02E3908033C031DF02E3808E83CB3
:100DE000031C8E2C3808E0003908E100172320305E
:100DF000E00016246E30E00016247330E000162464
:100E00002030E00016242030E00016242030E000DE
:100E100016242030E00016242030E0001624203074
:100E2000E00016242030E00016248E2CD5308312EA
:100E30000313A000C430A100BB30A200DC30A3002B
:100E4000A401A501A601A701A801A901AA01AB015E
:100E5000AC01AD01AE01AF01D201D301CB01CC0198
:100E6000D401D501D601D701B001B101B201B3015E
:100E7000D001D101CF018A110A12822C83120313EF
:100E80004A0E8400490E8A00480E8300FF0E7F0E32
:020E9000090057
:02400E00013F70
:00000001FF
